:100000000C94BC000C94D9000C94D9000C94D90029
:100010000C94D9000C94D9000C94D9000C94D900FC
:100020000C94D9000C94D9000C94D9000C94D900EC
:100030000C94D9000C94D9000C94D9000C94D900DC
:100040000C94B4010C94D9000C94D9000C94D900F0
:100050000C94D9000C94D9000C94D9000C94D900BC
:100060000C94D9000C94DB000C94D9000C94D900AA
:100070000C94D9000C94D9000C94D9000C94D9009C
:100080000C94D9000C94D9000C94D9000C94D9008C
:100090000C94D9000C94D9000C94D9000C94D9007C
:1000A0000C94D9000C94D9000C94D9000C94A9019B
:1000B0000C94D9000C94D9000C94D9000C94D9005C
:1000C0000C94D9000C94D9000C94D9000C94D9004C
:1000D0000C94D9000C94D9000C94D9000C94D9003C
:1000E0000C94D9000C94D9000C94D9000C94D9002C
:1000F0000C94D9000C94D9000C94D9000C94D9001C
:100100000C94D9000C94D9000C94D9000C94D9000B
:100110000C94D9000C94D9000C94D9000C94D900FB
:100120000C94D9000C94D9000C94D9000C94D900EB
:100130000C94D9000C94D9000C94D9000C94D900DB
:100140000C94D9000C94D9000C94D9000C94D900CB
:100150000C94D9000C94D9000C94D9000C949608F6
:100160000C94D9000C94D9000C94D9000C94D900AB
:100170000C94D9000C94D90011241FBECFEFDFE2FC
:10018000DEBFCDBF11E2A0E0B0E2ECEFF6E102C0CD
:1001900005900D92AC31B107D9F713E2ACE1B1E2B1
:1001A00001C01D92AB39B107E1F70E94FD060C9426
:1001B0007C0B0C949A011F920F920FB60F92112490
:1001C0008F939F93EF93FF9390918D218091A0083F
:1001D000EFE8F1E2E90FF11D808380918D218832F3
:1001E00030F480918D218F5F80938D2102C0109219
:1001F0008D2180916221883228F4809162218F5F65
:1002000080936221FF91EF919F918F910F900FBE8C
:100210000F901F90189580916221089590918C21E4
:10022000EFE8F1E2E90FF11D8081983220F49F5F41
:1002300090938C2102C010928C219091622199237D
:1002400029F0909162219150909362210895E0EA03
:10025000F8E0218125FFFDCF70E0E0E0F1E064A34C
:1002600075A3282F392F80A7C901AA2797FDA0952C
:10027000BA2F292F3A2F4B2F552721A7CD01AA2777
:10028000BB2782A780A1806880A30895E0EAF8E0F8
:10029000A0E0B1E0218125FFFDCF14962C911497A9
:1002A00025FDF8CF70E0E0E0F1E064A375A3282F0E
:1002B000392F80A7C901AA2797FDA095BA2F292F0A
:1002C0003A2F4B2F552721A7CD01AA27BB2782A75D
:1002D00080A1806880A30895E0E0F1E084E080A33D
:1002E00011A280E182A38CE483A316A280EA84A7F2
:1002F00088E085A716A6089510928C2110928D2172
:1003000010926221E0EAF8E080E3838388E184834D
:1003100083E085838FE1868380EE87830895E0EA1A
:10032000F8E0918195FF04C08093A00880E00895D3
:1003300081E008951F920F920FB60F9211248F93B0
:1003400081E0809396238F910F900FBE0F901F90A6
:1003500018951F920F920FB60F92112400000F9064
:100360000FBE0F901F9018951F920F920FB60F920D
:1003700011242F933F934F935F936F937F938F93AA
:100380009F93AF93BF93EF93FF938091B821909188
:10039000B9216CE040E00E942709FF91EF91BF91E5
:1003A000AF919F918F917F916F915F914F913F910D
:1003B0002F910F900FBE0F901F90189583E8809398
:1003C0000001089560E080E190E26F5FFC01E60FBC
:1003D000F11D20812223C9F780E190E20E942701CC
:1003E0000895EF92FF920F931F93CF93DF93FC0139
:1003F000CA012081243609F053C12BE320933F2109
:1004000020E22093402120934121209342212093F8
:10041000432120934421209345212093462120937A
:1004200047212091002020934821209101202093F2
:1004300049212091022020934A21209103202093DA
:100440004B212181223309F470C0233330F420334F
:1004500071F0213309F026C139C0243309F4C3C037
:10046000243308F491C0253309F01CC1EBC0FA0114
:10047000E60FF11D20E2208360E070E040E150E0F3
:100480000E94DB097B018C0180E0E81680E1F80620
:1004900080E0080780E0180708F006C1CFE3D1E24A
:1004A000BE016F5F7F4FC70140E150E00E94F30A39
:1004B000CE016DE00E942701C70160E00E9497090C
:1004C000E0920420F092052080E0F9C0FA01E60FE6
:1004D000F11D20E2208360E070E040E150E00E94E6
:1004E000DB097B018C0180E0E81680E1F80680E002
:1004F000080780E0180708F0D9C0CFE3D1E2BE01B9
:100500006F5F7F4FC70140E150E00E94F30ACE01C8
:100510006DE00E942701C70161E00E949709E09207
:100520000620F092072080E0CAC0FA01E60FF11D14
:1005300020E2208360E070E040E150E00E94DB09AF
:100540007B018C0180E0E81680E1F80680E0080776
:1005500080E0180708F0ACC0CFE3D1E2BE016F5FC6
:100560007F4FC70140E150E00E94F30ACE016DE0E9
:100570000E942701C70162E00E949709E0920820CB
:10058000F092092080E09BC0FA01E60FF11D20E205
:10059000208360E070E040E150E00E94DB097B01D5
:1005A0008C0180E0E81680E1F80680E0080780E032
:1005B000180708F07FC0CFE3D1E2BE016F5F7F4F25
:1005C000C70140E150E00E94F30ACE016DE00E94B5
:1005D0002701C70163E00E949709E0920A20F09288
:1005E0000B2080E06CC0FA01E60FF11D20E22083B1
:1005F00060E070E040E150E00E94DB097B018C018B
:1006000080E0E81680E1F80680E0080780E018073F
:1006100008F052C0CFE3D1E2BE016F5F7F4FC70148
:1006200040E150E00E94F30ACE016DE00E942701F4
:10063000C70164E00E949709E0920C20F0920D201F
:1006400080E03DC0FA01E60FF11D20E2208360E06A
:1006500070E040E150E00E94DB097B018C0180E00A
:10066000E81680E1F80680E0080780E0180730F51A
:10067000CFE3D1E2BE016F5F7F4FC70140E150E0A1
:100680000E94F30ACE016DE00E942701C70165E0D8
:100690000E949709E0920E20F0920F2080E00FC098
:1006A00081E00DC081E00BC081E009C081E007C09E
:1006B00081E005C081E003C081E001C081E0DF91FD
:1006C000CF911F910F91FF90EF900895FF920F939C
:1006D0001F93DF93CF93CDB7DEB7A297CDBFDEBF19
:1006E0008B01F22E89A39AA318A228A14F2D50E0C6
:1006F000332727FD30952417350794F460E3E8A1EC
:10070000FF27E7FDF095E00FF11F608328A12F5F21
:1007100028A328A1332727FD3095241735077CF31C
:10072000909581959F4FBE016F5F7F4F40E150E0F4
:100730000E94F30A1F8E8F8D8D31C0F48F8DFE01C4
:10074000E80FF11D8181882349F410C02F8DFC0131
:10075000E20FF11D2081222319F408C0CE01019679
:100760002F8D2F5F2F8F2F8D2D3180F38F8DF816CA
:1007700070F18F8D882359F18F8DF81A18A228A156
:100780008F8D332727FD309590E028173907FCF42B
:100790000F0D111DAE014F5F5F4FE8A1A8A1FF270C
:1007A000E7FDF095E00FF11FBB27A7FDB095A40F63
:1007B000B51F8C91808388A18F5F88A328A18F8D1E
:1007C000332727FD309590E02817390734F3A29698
:1007D000CDBFDEBFCF91DF911F910F91FF900895A4
:1007E0001F93CF93DF93FC0180818336A1F0843681
:1007F00030F48F3341F0813609F0E3C1C7C084364D
:1008000009F0DFC117C081818F3309F0DCC10E947C
:10081000E20180E0E1C18181843729F481E08093A5
:10082000FF2280E0D9C1863609F0CFC11092FF22A5
:1008300080E0D2C18BE380931C2180E380931D2153
:1008400088E780931E2180E280931F2180932021DE
:10085000809321218093222180932321809324213E
:100860008091002080932521809101208093262172
:10087000809102208093272180910320809328215A
:1008800081818233B9F1833330F4803369F081336D
:1008900009F09DC11CC0843309F452C08433E8F1CF
:1008A000853309F094C15FC0CCE1D1E2BE016D5F38
:1008B0007F4F809104209091052040E150E00E94FC
:1008C000F30ACE016DE00E94270180E085C1CCE1F2
:1008D000D1E2BE016D5F7F4F80910620909107208D
:1008E00040E150E00E94F30ACE016DE00E94270132
:1008F00080E072C1CCE1D1E2BE016D5F7F4F80919B
:1009000008209091092040E150E00E94F30ACE01B6
:100910006DE00E94270180E05FC1CCE1D1E2BE0121
:100920006D5F7F4F80910A2090910B2040E150E055
:100930000E94F30ACE016DE00E94270180E04CC1C5
:10094000CCE1D1E2BE016D5F7F4F80910C20909190
:100950000D2040E150E00E94F30ACE016DE00E94BC
:10096000270180E039C1CCE1D1E2BE016D5F7F4F4C
:1009700080910E2090910F2040E150E00E94F30AF8
:10098000CE016DE00E94270180E026C18BE38093B9
:100990001C2180E380931D2188E780931E2180E243
:1009A00080931F21809320218093212180932221F5
:1009B00080932321809324218091002080932521FE
:1009C000809101208093262180910220809327210D
:1009D000809103208093282181818233C9F1833360
:1009E00040F4803379F0813300F58A3209F0F1C0A8
:1009F0007BC0843309F452C08433E8F1853309F0B5
:100A0000E8C05FC0CCE1D1E2BE016D5F7F4F809155
:100A100002239091032340E150E00E94F30ACE01AB
:100A20006DE00E94270180E0D7C0CCE1D1E2BE0199
:100A30006D5F7F4F809104239091052340E150E04A
:100A40000E94F30ACE016DE00E94270180E0C4C03D
:100A5000CCE1D1E2BE016D5F7F4F80910623909182
:100A6000072340E150E00E94F30ACE016DE00E94AE
:100A7000270180E0B1C0CCE1D1E2BE016D5F7F4FC4
:100A8000809108239091092340E150E00E94F30AED
:100A9000CE016DE00E94270180E09EC0CCE1D1E252
:100AA000BE016D5F7F4F80910A2390910B2340E13F
:100AB00050E00E94F30ACE016DE00E94270180E021
:100AC0008BC0CCE1D1E2BE016D5F7F4F80910C23E2
:100AD00090910D2340E150E00E94F30ACE016DE0B9
:100AE0000E94270180E078C00E940509882309F44C
:100AF00072C0CCE1D1E28AE080931C21BE016F5F1D
:100B00007F4F809102239091032340E124E00E94D3
:100B1000660310E210932121BE016A5F7F4F80912E
:100B200004239091052340E124E00E946603109382
:100B30002621BE01655F7F4F809106239091072398
:100B400040E124E00E94660310932B21BE01605F08
:100B50007F4F809108239091092340E124E00E9477
:100B6000660310933021BE016B5E7F4F80910A2394
:100B700090910B2340E124E00E94660310933521FD
:100B8000BE01665E7F4F80910C2390910D2340E162
:100B900024E00E9466038091002080933A21809196
:100BA000012080933B218091022080933C21809101
:100BB000032080933D21CE0162E20E94270180E064
:100BC0000BC081E009C081E007C080E005C081E082
:100BD00003C081E001C080E0DF91CF911F910895B3
:100BE000909160219130D1F0913030F0923041F10C
:100BF000933009F064C040C0109253218D3011F041
:100C00008A3031F480E090E264E00E942701089588
:100C100080935E2181E08093602108958D3011F0F2
:100C20008A3041F41092602180E090E264E00E94FA
:100C30002701089580935F2182E0809360210895C9
:100C40008032B1F08D3011F08A3051F48EE591E2AE
:100C50000E94F00380E090E264E00E94270105C05A
:100C600080E090E264E00E942701109260210895E4
:100C700083E08093602108958D3011F08A3091F4E3
:100C8000109260218EE591E26091532144E551E29A
:100C90000E94F1018823D1F080E090E264E00E949C
:100CA00027010895909153219A3080F4E4E5F1E210
:100CB000E90FF11D80839F5F909353210895109257
:100CC000602180E090E264E00E9427010895DF93B4
:100CD000CF9300D0CDB7DEB7E82FF92FA62FB72FCF
:100CE00040E0308120E08181B901680F711D698386
:100CF0007A8389819A8195FF06C089819A81906C57
:100D000089839A8305C089819A819F7389839A8395
:100D100089819A818D939D934F5F3296463009F772
:100D20000F900F90CF91DF910895E0E0F6E01082F0
:100D300021E0218382E0818393E09483E0E2F6E086
:100D400010821482E0E4F6E010828483818398E0CC
:100D5000918335893061358BE0E6F6E0108221839E
:100D6000818334E03183918340E1418340E24183D8
:100D700040E8418341E1448343894068438BE0E894
:100D8000F6E0108221838183318391831482089558
:100D9000E0E5F0E08BEC8283808188608083E1E590
:100DA000F0E0808183FFFDCFE0E5F0E082EC858319
:100DB000808180618083E1E5F0E0808184FFFDCF68
:100DC00088ED84BF84E080934000E0E5F0E080811E
:100DD00080830895E0E0F8E085E0808381E181830D
:100DE00012821382148288EE93E080A791A783EF8A
:100DF0008487168283E0878308952F923F924F92D3
:100E00005F926F927F928F929F92AF92BF92CF929A
:100E1000DF92EF92FF920F931F93DF93CF93CDB7A3
:100E2000DEB7E797CDBFDEBFCE0101968093B82134
:100E30009093B9210E94950600E016E0FF24689483
:100E4000F1F8D8011596FC92159781E015968C93D0
:100E50000E94C8060E947C010E946C0188ED84BF3C
:100E6000E0E8F0E080818D7F8083E0E4F6E0F582C9
:100E7000E0EAF0E08281856082830E94BE090E94E0
:100E8000CB0978948FEF99EFA0E081509040A0407B
:100E9000E1F700C000000E94EA060E94DE01D801CE
:100EA0001696FC9280E090E264E00E942701109286
:100EB000FF220F2EF2E0CF2EF3E2DF2EF02D0F2EC9
:100EC000FDE0EF2EF02D0F2EFDE08F2E9924F02D5A
:100ED0008C0E9D1E0F2EFEE06F2E7724F02D6C0ED3
:100EE0007D1EFF246894F5F844245524689441F845
:100EF0004C0C5D1C0F2EF3E12F2E3324F02D2C0E05
:100F00003D1EF6013496E8ABF9ABC60106968AABF6
:100F10009BABD6011896ACABBDABF6013A96EEABE7
:100F2000FFAB0F2EF0E4AF2EF6E0BF2EF02D0E94A7
:100F30000B01882321F00E940E010E94F0050E94FF
:100F4000FC08882309F470C00E940809009709F082
:100F50006BC00E94FF08882309F066C00E94F90850
:100F6000B6010E9467060E940F0981E00E940209F3
:100F70008091FF22882331F4D50118968C9118971F
:100F800085FF4CC081E0F8018683ED86D6018D9106
:100F90009C91B30140E124E00E946603FA8AF201C9
:100FA00080819181B10140E124E00E946603FF8AC3
:100FB000A8A9B9A98D919C91BE01685E7F4F40E1BF
:100FC00024E00E946603FC8EEAA9FBA9808191813E
:100FD000BE01635E7F4F40E124E00E946603F9A2F8
:100FE000ACA9BDA98D919C91BE016E5D7F4F40E182
:100FF00024E00E946603FEA2EEA9FFA980819181F0
:10100000BE01695D7F4F40E124E00E946603FAE083
:10101000FBA7C4016FE10E94270108C081E0D8014D
:1010200015968C93159702C00E940F098091962304
:10103000882309F47CCF81E0F801858378CFFC0117
:10104000DB01213081F0213020F0223009F06DC029
:1010500056C0442309F469C080E091919D938F5F4D
:101060008417D8F308958181869586958C93918114
:10107000992314F4806C8C9391819295990F990F18
:10108000907C808186958695892B11968C931197FB
:1010900083818695869512968C93129793819923D6
:1010A00024F4806C12968C93129793819295990FE9
:1010B000990F907C828186958695892B13968C93C7
:1010C000139785818695869514968C9314979581B0
:1010D000992324F4806C14968C931497958192959F
:1010E000990F990F907C848186958695892B15960A
:1010F0008C931597868116968C9316970895808108
:101100008C93818111968C931197848112968C9384
:101110001297858113968C931397828114968C93E2
:101120001497838115968C93159708951F920F92AB
:101130000FB60F9211248F939F93EF93FF9388E044
:10114000E0E6F6E08683E0ECF9E0838190911821F7
:10115000E7EFF0E2E90FF11D8083809118218E31D5
:1011600028F4809118218F5F809318218091172196
:1011700081508093172180911721882339F581E0D0
:10118000809315211092192180911A2190911B2191
:10119000009781F4E0ECF9E080818F7B808380E828
:1011A000E0E6F6E08583E0E0F9E082E0808381819B
:1011B0008061818380911A2190911B21813091055A
:1011C00079F480E1E0E6F6E085830AC08091182199
:1011D000E7EFF0E2E80FF11D8081E0ECF9E08383B6
:1011E000FF91EF919F918F910F900FBE0F901F90E5
:1011F000189587EF90E208958091152108958091C8
:101200001921089580931921089580911621089538
:1012100020911A2130911B21822F932F08958091C4
:101220001521882319F081E0809316210895E0E0CC
:10123000F9E082E0808381E181831282138214824B
:101240001682178282E090E080A791A70895FF920E
:101250000F931F93F82E092F162F809116218823A4
:1012600009F45CC06E3108F05BC010921621109238
:101270001521842F90E080931A2190931B21609375
:10128000172110921821E0ECF9E0808180648083BE
:10129000442319F0413019F525C0E0E0F9E010824F
:1012A00081818F7E818381E0E0E6F6E08683809114
:1012B0006121882329F40E94170981E0809361212C
:1012C000E0ECF9E089E5808383E08183E0E6F6E005
:1012D00088E08583000081E08683000085831123F8
:1012E00041F415C0E0ECF9E08DED808383E081836B
:1012F000F6CFEF2DF02F80E090E027EF30E2419124
:10130000D901A80FB91F4C9301968117C0F38091A2
:10131000F720E0ECF9E0838380E003C082E001C0C5
:1013200081E01F910F91FF90089581E00895DF9370
:10133000CF9300D00F92CDB7DEB76730C0F46063B3
:1013400069839C01329522952F7023273F702327B4
:101350002A838295807F8B8380E1E0E6F6E08683B6
:10136000CE01019663E041E00E94270901C081E0BF
:101370002396CDBFDEBFCF91DF910895E0E6F6E082
:1013800080EB818380E1858386E0818382E08583B1
:1013900084E085830895E0E6F6E089E0818388E0D3
:1013A000868391E09583E0E8F6E09FE0918395E005
:1013B0009583858308952F923F924F925F926F920B
:1013C0007F929F92AF92BF92CF92DF92EF92FF9265
:1013D0000F931F93CF93DF933B01EA0161157105D2
:1013E00019F0FB0180839183209739F09E012250F0
:1013F00030402332310508F0D7C0C82ED92EF6016F
:1014000011916F017F01812F90E00E94EB0A0097FC
:10141000B1F71D3231F4F60111917F0199249394B3
:1014200006C01B3219F4F60111917F01992420970F
:1014300019F0C031D105D1F4103389F4F70180815E
:10144000883711F0883559F4F701118182E090E076
:10145000E80EF91E92E0992AC0E1D0E007C020977B
:1014600029F41033B1F0CAE0D0E02CC0CA30D10565
:1014700049F1C031D10521F0C830D105A9F409C026
:101480002FEFA22E2FEFB22E2FEFC22E2FE0D22E53
:1014900021C0C8E0D0E09FEFA92E9FEFB92E9FEFAB
:1014A000C92E9FE1D92E16C09E01442737FD4095D5
:1014B000542F6FEF7FEF8FEF9FEF0E945A0B590170
:1014C0006A0108C089E9A82E89E9B82E89E9C82EE1
:1014D00089E1D82E60E020E030E0A9011E0144241B
:1014E00037FC4094542C012F00530A3060F0812FB8
:1014F00081548A3110F4075006C0812F81568A31F9
:1015000050F5012F0755802F90E08C179D071CF593
:101510006F3FE9F0A216B306C406D506A8F0CA01CB
:10152000B901A20191010E94270B9B01AC01802F00
:1015300090E0A0E0B0E0280F391F4A1F5B1F28177A
:1015400039074A075B0710F46FEF01C061E0F7014C
:1015500011917F01C8CF6114710481F0662339F0C5
:101560000894E108F108F301E082F18207C091FEDE
:1015700005C0C7010297F3018083918390FE07C0E5
:1015800050954095309521953F4F4F4F5F4F67FFE6
:101590000EC082E290E08093992390939A232FEFDC
:1015A0003FEF4FEF5FEF03C020E030E0A901B9014A
:1015B000CA01DF91CF911F910F91FF90EF90DF90C3
:1015C000CF90BF90AF909F907F906F905F904F9023
:1015D0003F902F900895911127C0803219F08950C3
:1015E0008550D0F70895FB019F01E8944230C4F084
:1015F0004532B4F44A3029F497FB1EF49095819556
:101600009F4F642F77270E94460B805D8A330CF032
:10161000895D8193CB010097A1F716F45DE25193A8
:101620001082C9010C94170B992788270895DC01B3
:10163000FC01672F71917723E1F7329704C07C9109
:101640006D9370836291AE17BF07C8F30895629FD0
:10165000D001739FF001829FE00DF11D649FE00DAA
:10166000F11D929FF00D839FF00D749FF00D659F0B
:10167000F00D9927729FB00DE11DF91F639FB00D0A
:10168000E11DF91FBD01CF0111240895AA1BBB1B49
:1016900051E107C0AA1FBB1FA617B70710F0A61B72
:1016A000B70B881F991F5A95A9F780959095BC0193
:1016B000CD010895A1E21A2EAA1BBB1BFD010DC08E
:1016C000AA1FBB1FEE1FFF1FA217B307E407F507F2
:1016D00020F0A21BB30BE40BF50B661F771F881FCE
:1016E000991F1A9469F760957095809590959B0164
:0C16F000AC01BD01CF010895F894FFCFBC
:1016FC000A0D3A3EFF07FF07FF07FF07FF07FF072B
:10170C000A0D2A2A2A2056455253494F4E20393960
:10171C002E3939202A2A2A0A0D202D20613C302D01
:10172C00353E3A20646973706C61792041444320E2
:10173C0076616C75650A0D202D20643C302D353E8C
:10174C003A20646973706C6179204441432076615E
:10175C006C75650A0D202D20643C302D353E203CE7
:10176C006865782076616C75653E3A2073657420E7
:10177C004441432076616C75650A0D202D20733C25
:10178C00737C6D3E3A2073796E63207065722073A2
:10179C00616D706C65207C206D6561737572656D13
:1017AC00656E740A0D202D203F3F202020203A200A
:1017BC0053686F7720696E666F200A3A3E0A0D20D7
:1017CC002D20633C747C663E3A20436F6E74696EC8
:1017DC00756F757320646174612074727565207CFB
:1017EC002066616C736500000000000000000000C2
:1017FC0000000000000000000000000000000000DD
:0C180C00000000000001010000010000CD
:00000001FF
